:0200000480007A
:100000006F00C0006F20802C6F20402C93000000F8
:10001000130100009301000013020000930200008E
:100020001303000093030000130400009304000076
:10003000130500009305000013060000930600005E
:100040001307000093070000130800009308000046
:100050001309000093090000130A0000930A00002E
:10006000130B0000930B0000130C0000930C000016
:10007000130D0000930D0000130E0000930E0000FE
:10008000130F0000930F000097020000938202F804
:100090007390523017B100001301C1E4F32240F114
:1000A0009392C2003301510073100134EF20900B82
:1000B000173500001305858B6F20006B8332851088
:1000C000739012148330850003310501833185015B
:1000D000033205028332850203330503833385032C
:1000E000033405048334850483358505033605060A
:1000F00083368506033705078337850703380508E8
:10010000833885080339050983398509033A050AC7
:10011000833A850A033B050B833B850B033C050CA7
:10012000833C850C033D050D833D850D033E050E87
:10013000833E850E033F050F833F850F033505057D
:10014000730020107311011423341100233C31007B
:10015000233041022334510223386102233C7102CF
:1001600023308104233491042338A104233CB104B7
:100170002330C1062334D1062338E106233CF1069F
:10018000233001092334110923382109233C310983
:100190002330410B2334510B2338610B233C710B6B
:1001A0002330810D2334910D2338A10D233CB10D53
:1001B0002330C10F2334D10F2338E10F233CF10F3B
:1001C000F312011423385100F32200102330511090
:1001D000F322101423345110F32230142338511019
:1001E000F3222014233C5110130501006F208033AB
:1010000000000000000000000000000000000000E0
:1010100000000000000000000000000000000000D0
:1010200000000000000000000000000000000000C0
:1010300000000000000000000000000000000000B0
:081040000000000000000000A8
:10200000B367B500B3E7C70093F77700B306C50021
:10201000638407023386C50093070500637ED502FB
:1020200003C705009385150093871700A38FE7FE6C
:10203000E398C5FE67800000E37ED5FE93070500A8
:1020400003B70500938787009385850023BCE7FECF
:10205000E3E8D7FE6780000067800000130101FFFE
:10206000B367C500233081002334110093F7770054
:10207000130405003307C500638207026376E50099
:1020800093F5F50FEFF09FFD8330810013050400F9
:1020900003340100130101016780000093F5F50F7F
:1020A00093968500B3E6B60093970601B3E7D70091
:1020B00093960702B3E6F600E378E5FC9307050084
:1020C0009387870023BCD7FEE3ECE7FE83308100D3
:1020D00013050400033401001301010167800000AF
:1020E00083470500638E07009307050003C71700A9
:1020F00093871700E31C07FE3385A7406780000025
:1021000013050000678000008347050093851500D4
:102110001305150003C7F5FF638A0700E386E7FE92
:102120001B8507003B05E5406780000013050000A4
:102130006FF05FFFB367B50093F77700639E070208
:10214000137886FF330805016378050393070500BC
:102150006F000001938787009385850063F807016E
:1021600083B6070003B70500E386E6FE3385A74084
:102170003306A640138507003386C5006F00400173
:1021800003C705008347F5FF93851500639AE700B1
:1021900013051500E396C5FE1305000067800000D7
:1021A0003B85E740678000009307050003C70500F3
:1021B0009387170093851500A38FE7FEE31807FEAA
:1021C000678000000347050093060002930705009F
:1021D0006318D70003C7170093871700E30CD7FED7
:1021E0009306D0026300D7069306B0026300D704BB
:1021F00083C60700930500006382060413050000F0
:1022000093871700131725001B8606FD83C607005A
:102210003307A700131717003305E600E39206FE05
:10222000638005023305A0406780000083C6170065
:102230009305000093871700E39206FC1305000046
:102240006780000083C6170093051000938717006E
:10225000E39606FA130500006FF09FFE8347050022
:10226000638007049305101017F7FFFF130787D942
:10227000939505030336070013051500B3E6B70071
:10228000630A060097F7FFFF23BE07DA83370700CC
:10229000E39A07FE2330D70083470500E39C07FC41
:1022A0006780000017F7FFFF1307C7D583370700C4
:1022B000638A070097F7FFFF23B607D88337070025
:1022C000E39A07FE2330A7006F000000130101FF0F
:1022D0001305903423341100EFF0DFFC130101FEED
:1022E0001306810093077101130890006F008000AE
:1022F000930707009376F500138706009305000304
:102300006374D800930570053B07B7002380E7008E
:10231000135545001387F7FFE31CF6FC8347810044
:10232000230C0100638207041305101093060600B6
:1023300017F7FFFF130707CD1315050383350700B4
:102340009386160033E6A700638A050097F7FFFF20
:1023500023BA07CE83370700E39A07FE83C7060038
:102360002330C700E39C07FC1301010267800000D3
:10237000130101FF37F8FFFF233411003307050174
:10238000B7E703006378F7141357C5009306076097
:1023900017460000130606C793973600B307F600EA
:1023A00083B70700337505016390070E978500001A
:1023B0009385C5C503B805006302081483378800F8
:1023C0009788000083B808C423B0F500638E170F08
:1023D0008337080093983600B308160193D7C700D7
:1023E0009397A70013E3F70D93E5F70123B0680077
:1023F00073000512973700009387C7C01317470073
:10240000B387E70003B7070063140710033708001A
:10241000B708040023B0E7000337880023B4E700BF
:10242000F3A80810B707E0FFB307F500371800005E
:10243000130705003388070103BF070083BE870029
:1024400003BE070103B387012330E7012334D7011B
:102450002338C701233C670093870702130707024D
:10246000E39C07FD7390081093973600B306F600BF
:1024700023B0B600730005120F10000083308100F6
:10248000130101016780000013F70704630A0702C4
:1024900013F70708631A07041307F00093E7070808
:1024A0006394E50493963600B306D60023B0F60095
:1024B0007300051283308100130101016780000061
:1024C00093E707046FF01FFE9787000023BC07B255
:1024D0006FF01FF017150000130545AFEFF01FD880
:1024E00013053000EFF01FDC17150000130585B24F
:1024F000EFF0DFD613053000EFF0DFDA171500003C
:102500001305C5B5EFF09FD513053000EFF09FD947
:1025100017150000130505B6EFF05FD41305300062
:10252000EFF05FD883358511130101F82338810658
:10253000233C11062334910623302107233C310527
:10254000233841052334510523306105233C7103B1
:1025500023388103233491032330A103233CB101A9
:102560009307800013040500638AF50E930720008B
:102570006380F506938745FF130710006376F70025
:102580009307F0006392F51A03350411EFF05FDE54
:102590001305040003340107833081078334810667
:1025A0000339010683398105033A0105833A810421
:1025B000033B0104833B8103033C0103833C810211
:1025C000033D0102833D8101130101086FD01FAF5C
:1025D000033785109377370063980706EF0780006D
:1025E000731030000327070083A70700630AF7046E
:1025F000130510109307100497160000938686ABFE
:1026000017F7FFFF130707A013150503833507000E
:102610009386160033E6A700638A050097F7FFFF4D
:1026200023B207A283370700E39A07FE83C7060099
:102630002330C700E39C07FC13053000EFF09FC672
:1026400013051000EFF01FC617150000130585B025
:10265000EFF0DFC013053000EFF0DFC403290505FC
:10266000371C0000973400009384C499974B0000F6
:10267000938B4B99370B0400B70AE0FF978D00004E
:10268000938D4D98178A0000130A4A98B7F90300F2
:102690006F0080012334F70023B0FD00B71700005E
:1026A000330CFC00630E3C0B9357CC001394470093
:1026B0003387840003370700E30207FE9387076030
:1026C00093973700B387FB0083BC070093F70C0494
:1026D000638E0706732D0B1037160000B3055C01DF
:1026E00013050C002334B100EFF0DFA4630E0500E6
:1026F00093FC0C088335810063800C0437160000BE
:1027000013050C00EFF0DF8FB387840073100D10FA
:1027100003B70D0023B00700E31E07F623B0FD004A
:102720002330FA006FF09FF717150000130505A579
:10273000EFF0DFB26FF05FF0171500001305059E94
:10274000EFF0DFB113053000EFF0DFB51715000033
:1027500013054599EFF09FB013053000EFF09FB4DB
:1027600013050900EFF01FB4F32740F1639A07182F
:102770009767000093870789130101ED93D7C7007E
:1027800023308112177800001308C887130405004E
:102790009397A700175500001305C586233411121F
:1027A0009356C5001357C80093E7170097480000D9
:1027B000938848851306F0FF233CF5FE9396A60008
:1027C0001317A700B707002093E61600136717003A
:1027D00093D5C8001313F6039387F70C233CF8FE38
:1027E00023B0D8002330E500B3E7650073900718E5
:1027F00073270018639EE7141356B6009307F00181
:102800009702000093824201F39252307310063B0C
:102810007390073A739052301308F0BF13185801A1
:1028200097E7FFFF93874792B3870701739057108D
:10283000F3270034B387070173900714B7B700007C
:102840009B87071073902730B7E701009B870760CD
:10285000739007307350403017370000130787B963
:102860009307083EB3060701B307F700B70808004F
:1028700017760000233CD67817330000130383F645
:102880009776000023B0F6789388F8039307A000AA
:102890001308080113D61700B3861701B347F600D3
:1028A000B30507019396C600939757002330D700CE
:1028B0002334B70093F7070213070701B367F60045
:1028C000E31AE3FC13060012930500001305010050
:1028D0009737000023B407F0EFF04FF8B7070080F8
:1028E0003304F4001305010023348110EFD00FFDF1
:1028F0008330811203340112130101136780000039
:1029000013071000B7476B0337060800938757C8B3
:102910001306C6FF1315F7019316E7036F00C001F6
:102920002F20070013D71700B3C7E7009397E703DB
:10293000B3F7D700B3E7E70033F7C70093F5170005
:102940003307A700E39E05FC032007006FF09FFDFF
:102950001715000013058585EFF05F901305300013
:10296000EFF05F946780000097100000938080690B
:10297000370155001B0151051311010113015105C8
:10298000131111011301A10A23B0200003B70000A5
:10299000B70355009B83530593930301938353051A
:1029A000939313019383A30A93012000631077602C
:1029B00097100000938000653701D5FF1B0151057A
:1029C00013110101130151051311D1001301B100BD
:1029D0001311C100130101A023B4200003B780002C
:1029E000B703D5FF9B83530593930301938353054B
:1029F0009393D3009383B3009393C300938303A073
:102A0000930130006314775A971000009380805F21
:102A1000370155001B0151051311D1001301B100FD
:102A20001311C100130111A01311C100130101AA58
:102A300023B8200003B70001B70355009B8353055B
:102A40009393D3009383B3009393C300938313A012
:102A50009393C300938303AA9301400063187754B0
:102A6000971000009380005A3701FDFF1B015105AC
:102A70001311010113015105131101011301510536
:102A80001311D1001301A10023BC200003B7800162
:102A9000B703FDFF9B835305939303019383530572
:102AA00093930301938353059393D3009383A300DC
:102AB00093015000631C774E9710000093800058DC
:102AC000370155001B015105131101011301510577
:102AD000131111011301A10A23B420FE03B780FED4
:102AE000B70355009B8353059393030193835305C9
:102AF000939313019383A30A930160006318774AA9
:102B000097100000938080533701D5FF1B015105BA
:102B100013110101130151051311D1001301B1006B
:102B20001311C100130101A023B820FE03B700FF59
:102B3000B703D5FF9B8353059393030193835305F9
:102B40009393D3009383B3009393C300938303A021
:102B500093017000631C7744971000009380004E2F
:102B6000370155001B0151051311D1001301B100AC
:102B70001311C100130111A01311C100130101AA07
:102B800023BC20FE03B780FFB70355009B8353058A
:102B90009393D3009383B3009393C300938313A0C1
:102BA0009393C300938303AA93018000631077403B
:102BB00097100000938080483701FDFF1B015105ED
:102BC00013110101130151051311010113015105E5
:102BD0001311D1001301A10023B0200003B700009E
:102BE000B703FDFF9B835305939303019383530521
:102BF00093930301938353059393D3009383A3008B
:102C0000930190006314773A9710000093808043FB
:102C1000377124001B01D18A1311E100130191C007
:102C20001311D100130151341311C1001301816735
:102C3000138200FE2330220283B20000B773240007
:102C40009B83D38A9393E300938393C09393D3009E
:102C5000938353349393C300938383679301A000BA
:102C600063967234971000009380C03D3741B000E6
:102C70001B0111261311C1001301B1301311F10012
:102C8000130131211311C100130181099380D0FF79
:102C9000A3B52000171200001302423B833202004A
:102CA000B743B0009B8313269393C3009383B33041
:102CB0009393F300938333219393C3009383830906
:102CC0009301B0006394722E9301C00013020000C0
:102CD000B7D0BB0A9B80D0CD171100001301813201
:102CE0002330110003370100B7D3BB0A9B83D3CD38
:102CF000631E772A1302120093022000E31A52FC8B
:102D00009301D00013020000B7C0AB0A9B80D0CC67
:102D1000171100001301012F1300000023341100CC
:102D200003378100B7C3AB0A9B83D3CC63107728EA
:102D30001302120093022000E31852FC9301E000FA
:102D400013020000B7C0AA0D9B80C0BC1711000081
:102D50001301412B13000000130000002338110061
:102D600003370101B7C3AA0D9B83C3BC631077244B
:102D70001302120093022000E31652FC9301F000AC
:102D800013020000B7B0DA0D9B80C0BB1300000037
:102D90001711000013010127233C110003378101A3
:102DA000B7B3DA0D9B83C3BB631277201302120003
:102DB00093022000E31852FC93010001130200006B
:102DC000B7B0DD0C9B80B0AB130000001711000002
:102DD00013014123130000002330110203370102C5
:102DE000B7B3DD0C9B83B3AB6312771C13021200E5
:102DF00093022000E31652FC93011001130200001D
:102E0000B7E0CD0C9B80B0AA1300000013000000B7
:102E1000171100001301011F23341102033781022F
:102E2000B7E3CD0C9B83B3AA631277181302120089
:102E300093022000E31652FC9301200113020000CC
:102E4000171100001301011CB72011009B803023D3
:102E50002330110003370100B72311009B83332374
:102E6000631677141302120093022000E31A52FC37
:102E700093013001130200001711000013018118A3
:102E8000B71001309B803022130000002334110062
:102E900003378100B71301309B8333226318771007
:102EA0001302120093022000E31852FC9301400128
:102EB00013020000171100001301C114B7100033F2
:102EC0009B80201213000000130000002338110023
:102ED00003370101B71300339B8323126318770C68
:102EE0001302120093022000E31652FC93015001DA
:102EF00013020000171100001301C110130000009D
:102F0000B70030239B802011233C1100033781013F
:102F1000B70330239B832311631A7708130212002F
:102F200093022000E31852FC930160011302000099
:102F3000171100001301010D13000000B700332228
:102F40009B8010011300000023301102033701029F
:102F5000B70333229B831301631A77041302120011
:102F600093022000E31652FC93017001130200004B
:102F700017110000130101091300000013000000E5
:102F8000B73023129B8010002334110203378102D3
:102F9000B73323129B831300631A770013021200C6
:102FA00093022000E31652FC631A300013951100BF
:102FB0006300050013651500730000001305100081
:082FC00073000000731000C053
:102FC800417373657274696F6E206661696C6564BC
:102FD8003A2061646472203E3D202831554C203CE3
:102FE8003C203132292026262061646472203C204E
:102FF8003633202A202831554C203C3C20313229B8
:103008000A00000000000000417373657274696F64
:103018006E206661696C65643A20212870745B33A0
:103028005D5B616464722F2831554C203C3C203133
:1030380032295D2026203078303830292026262075
:103048006361757365203D3D203078660A00000095
:10305800417373657274696F6E206661696C65642B
:103068003A206E6F64650A00417373657274696F04
:103078006E206661696C65643A20757365725F6D70
:10308800617070696E675B616464722F2831554C9A
:10309800203C3C203132295D2E61646472203D3D24
:1030A80020300A0000000000417373657274696F74
:1030B8006E206661696C65643A202122696C6C65D2
:1030C80067616C20696E737472756374696F6E22C0
:1030D8000A00000000000000417373657274696F94
:1030E8006E206661696C65643A2070745B335D5B61
:1030F800616464722F2831554C203C3C20313229C0
:103108005D20262030783034300A000000000000AE
:10311800417373657274696F6E206661696C65646A
:103128003A2070745B335D5B616464722F2831559B
:103138004C203C3C203132295D2026203078303824
:10314800300A000000000000417373657274696FF3
:103158006E206661696C65643A2074662D3E657000
:103168006320252034203D3D20300A000000000067
:10317800417373657274696F6E206661696C65640A
:103188003A202122756E65787065637465642065E0
:103198007863657074696F6E220A00000000000091
:1031A800417373657274696F6E206661696C6564DA
:1031B8003A202122756E737570706F727465642081
:0C31C80073617470206D6F6465220A0052
:10400000EFBEADDEEFBEADDEEFBEADDEEFBEADDED0
:10401000EFBEADDEEFBEADDEEFBEADDEEFBEADDEC0
:10402000EFBEADDEEFBEADDEEFBEADDEEFBEADDEB0
:10403000EFBEADDEEFBEADDEEFBEADDEEFBEADDEA0
:10404000EFBEADDEEFBEADDEEFBEADDEEFBEADDE90
:040000058000000077
:00000001FF
